:1000000059C0FECFFDCFFCCFFBCFFACFF9CFF8CF51
:10001000F7CFF6CFF5CFF4CFF3CFF2CFF1CFF0CFCC
:06002000EFCFEECFEDCFA3
:1000B400BFE5BDBFB4E0BEBF2F92BEB5B160BEBD4B
:1000C400BEB5B260BEBDBEB5B460BEBDB0ECB7BB1C
:1000D400B0E0B4BBB0E4B1BBBFE3B8BBBFEFB5BBEA
:1000E400BFEBB2BBDADFB0E0BDBDB0E0BCBD25E024
:1000F4001FE002EF0A95F1F71A95E1F72A95D1F777
:100104000CB5009366000DB500936700B1E02B2E8B
:10011400BFDF009364001093650020E0322F46E4B3
:1001240050E060E070E096DFBAE0369527951795C9
:100134000795BA95D1F7065A1F4F2F4F3F4F00939B
:10014400600010936100209362003093630020915B
:1001540066003091670004E110E00217130708F00D
:1001640041C0B8B3B064B8BB409160005091610025
:100174006091620070916300425050406040704052
:10018400009166001091670020E0322F04171507D4
:100194002607370720F4B8B3B068B8BB03C0B8B3B8
:1001A400BF77B8BB0091600010916100209162009C
:1001B40030916300A801B9014E5F5F4F6F4F7F4FCD
:1001C400009166001091670040175107B0E06B077B
:1001D4007B0720F4B2B3B064B2BB03C0B2B3BF7B3D
:1001E400B2BB09C0B8B3BF7BB8BBB8B3BF77B8BBA9
:0C01F400B2B3BF7BB2BB77CF2F90FFCF20
:10009E00B6E1B0936800B0E0B0936900B7E8B6B9C6
:0600AE00B0E0B7B90895AF
:0A00940004D0CADF98018901089525
:10002C0007B1007E022907B9B6B1B064B6B9B6B152
:10003C00B6FF02C00000FBCF24B130E005B1102F99
:0C004C000027022B132B98018901089556
:10005800049FD001159FF001249FE00DF11D069F1C
:10006800E00DF11D349FF00D259FF00D169FF00D4A
:10007800079FF00D3327149FB00DE11DF31F059F57
:0C008800B00DE11DF31F8D019F010895D4
:00000001FF
